:100000000C9455010C9472010C9472010C947201C1
:100010000C9472010C9472010C9472010C94720194
:100020000C9472010C9472010C940F1D0C94E11D40
:100030000C9401180C9472010C9472010C947201CE
:100040000C9472010C9472010C9472010C94720164
:100050000C9472010C9489180C9472010C94720126
:100060000C9472010C9472010C9472010C94720144
:100070000C9472010C9472010C9472010C94720134
:100080000C9472010C9472010C9472010C94720124
:100090000C9472010C9472010C9472010C94720114
:1000A0000C9472010C9472010C94720122042204CB
:1000B0004E044E04B604D404EC05EC05DF047805C8
:1000C000890589054E1E751E6D1F751E6D1FC11E8B
:1000D000E41E6D1F3B1F4A1F0100530054005500D2
:1000E000560001005F0060006100570001005C00E5
:1000F0005D005E000000010059005A005B005800DE
:100100000000620000006300000001000100010027
:1001100001000100010001000100010001000100D7
:1001200001000100010001000100010001000100C7
:1001300001000000010001000100010012034E0057
:1001400075006D0062007200650072006F000000B3
:10015000100346006C0065006800720061006400D6
:1001600000000403090409023B00020100A0FA098F
:1001700004000001030101000921110100012240D6
:1001800000070581030800010904010001030000C4
:100190000009211101000122B60007058203200099
:1001A000011201000200000008EDFE606001000184
:1001B00002000105010902A10185020901A1000552
:1001C0000919012908150025019508750181020505
:1001D00001093009311581257F95027508810609CD
:1001E000381581257F950175088106050C0A3802AE
:1001F0001581257F950175088106C0C0050109801C
:10020000A101850319012AB700150126B700950140
:1002100075108100C0050C0901A101850419012A8E
:10022000A002150126A002950175108100C00501EC
:100230000906A1018506050719E029E71500250132
:100240009508750181020507190029EF15002501A0
:1002500095F07501810205081901290595057501BB
:100260009102950175039101C005010906A10105DF
:100270000719E029E7150025019508750181029508
:1002800001750881010507190029FF150026FF00E7
:100290009506750881000508190129059505750160
:1002A0009102950175039101C00011241FBECFEF8B
:1002B000DAE0DEBFCDBF11E0A0E0B1E0E0E4F0E4C1
:1002C00002C005900D92A638B107D9F722E0A6E842
:1002D000B1E001C01D92AE38B207E1F70E94CB1128
:1002E0000C941E200C94000081E0089581E0089594
:1002F0000C94760108950C947A011F93CF93DF93A9
:1003000000D000D01F92CDB7DEB749835A836B83EC
:100310003091890189819A81311114C0662359F085
:10032000222349F00E942B08182F682F89819A8177
:100330000E94D20703C00E94FE07182F69817A81AC
:10034000812F04C00E942B0869817A810F900F9041
:100350000F900F900F90DF91CF911F910C944C0F45
:10036000FC01262F408151816281738184810C942C
:100370007D0181E00895CF93DF93EC0160E00E945E
:10038000B001BE01DF91CF910C947B010C948F10D2
:100390000C948B1008950E947C060E94CA012FEFD6
:1003A00084E39CE0215080409040E1F700C00000D1
:1003B0000C94AF180F931F93CF93DF938C0161E0E0
:1003C0000E94B001EC01B8010E9478018823F1F18C
:1003D000B801CE010E944D168823C1F1B801CE01AB
:1003E0000E946114882391F1B801CE010E94A915E1
:1003F000882361F1F8018281882309F1CB358DE5ED
:10040000D807C1F050F4C115FCE5DF0781F0CF3DFE
:10041000DC45A9F40E94620D19C0CC35EDE5DE077C
:1004200061F0CD35DD4559F40E94A50C08C00E944D
:10043000CB010CC00E94AE0C02C00E94B10CC801DE
:10044000DF91CF911F910F910C94740180E0DF91A7
:10045000CF911F910F9108950E94E4170C944502CB
:100460000E9448020C94EA1708950C94340281E02B
:1004700008950C9437020895CF93C82F0E94350237
:100480008C2F0E943902CF91089580E00C943C0299
:100490000E94A9160C943C020E94A9169091880112
:1004A000891721F0809388010C943C020895CF9322
:1004B000DF93CDB7DEB72B970FB6F894DEBF0FBE34
:1004C000CDBF4F83588769877A878B8761110E94D8
:1004D000F10B9E012F5F3F4F86E0F90111928A9543
:1004E000E9F785E0FE013796D90101900D928A95D2
:1004F000E1F789819A814C815D81452B31F09F3FE5
:1005000031F491E08F3F19F403C091E001C090E015
:1005100090FF09C049815A816B817C818D819E81C8
:100520000E94120B05C0C9010E94B9018111F2CFCE
:100530002B960FB6F894DEBF0FBECDBFDF91CF91E3
:100540000895FC01808191810E946D080895CF93E8
:10055000882309F4A4C0C82F8238C1F40E94A916C8
:1005600081FD9DC069E380910201909103010E9489
:100570009F170E94130C2FEF81EE94E021508040D2
:100580009040E1F700C0000069E319C0833801F52D
:100590000E94A91680FD83C063E5809102019091BD
:1005A00003010E949F170E94130C2FEF81EE94E02D
:1005B000215080409040E1F700C0000063E5809149
:1005C0000201909103010E94AA17CF910C94130C81
:1005D0008438C1F40E94A91682FD61C067E480914D
:1005E0000201909103010E949F170E94130C2FEFAC
:1005F00081EE94E0215080409040E1F700C000007F
:1006000067E4DDCF8CEF8C0F813AD0F46C2F8091B2
:100610000201909103010E941F17882349F06C2F5B
:1006200080910201909103010E94AA170E94130C6D
:100630006C2F80910201909103010E949F17C5CFFA
:1006400080E28C0F883048F4C77081E001C0880FC9
:10065000CA95EAF70E94D40BB8CFEBE5EC0FE33074
:1006600040F4F0E0E95BFE4F808190E0CF910C9484
:10067000DD16E8E5EC0FE73150F4F0E0EE0FFF1F78
:10068000E75EFE4F80819181CF910C94F316CD3EB1
:1006900030F08C2F0E945012CF910C942213CF91E6
:1006A0000895882309F464C0823879F40E94A91659
:1006B00081FF5EC069E380910201909103010E9475
:1006C0009F170E94130C69E310C08338B1F40E9495
:1006D000A91680FF4DC063E580910201909103014E
:1006E0000E949F170E94130C63E580910201909174
:1006F00003010E94AA170C94130C843879F40E9409
:10070000A91682FF35C067E4809102019091030130
:100710000E949F170E94130C67E4E7CF9CEF980F8D
:10072000913A10F4682FE1CF90E2980F983050F48E
:10073000877091E001C0990F8A95EAF7892F0E948E
:10074000DA0BD9CF9BE5980F933020F480E090E04E
:100750000C94DD1698E5980F973120F480E090E036
:100760000C94F3168D3E20F00E94AB120C942213D1
:1007700008951F93CF93DF93182FEB010E94A702D8
:10078000209741F08FE99FE00197F1F700C000004A
:100790002197F6CF812FDF91CF911F910C945103B8
:1007A000893319F060E070E002C060E570E00C94FD
:1007B000B903882321F00E94D40B0C94130C0895E4
:1007C000882321F00E94DA0B0C94130C0895CF9229
:1007D000DF92EF92FF920F931F93CF93DF937C01F1
:1007E000D62FC72FFC011281058102950F700E9440
:1007F000CA0B8823B9F01123A9F08C2F807F803495
:1008000021F080E28D0F883068F08091720282FDC5
:1008100009C082E00E94730C0E94CA0B91E0D82E9E
:10082000D92601C0D12CCC2EC2948FE0C8228C2DA9
:1008300090E08C30910508F0CFC1FC01EA5AFF4FDF
:100840000C94B51F8C2F807FCF70882311F0C29538
:10085000C07F112399F0CC2309F4AAC180E28D0F47
:10086000883010F0D11104C08C2F0E94D40B03C02B
:100870008C2F0E94E40B0E94130C9AC18D2F0E94B2
:100880005103CC2309F4A8C180E28D0F883038F1E0
:10089000DD2329F18C2F0E94EA0B24C08C2F807F4E
:1008A000CF70803211F0C295C07FDD2319F0D130B6
:1008B000A1F13DC08091720282FF17C0112349F05F
:1008C000CC2329F08C2F0E94D40B0E94130C80E0C3
:1008D00070C180E00E945103CC2309F47DC18C2FAC
:1008E0000E94DA0B0E94130C77C1112371F00023D0
:1008F00041F0013031F40E94F40B8C2B0E94FC0B70
:100900006BC10E94F40B8C2B1DC0002319F0013029
:1009100009F462C10E94090C25C0112321F00630A0
:1009200008F05AC10EC0053008F056C11BC0112393
:1009300061F0002331F0F701858180FF39C18F70AC
:1009400085838C2F0E94D90347C1002359F0D933E6
:1009500009F03FC1FFEF07EE13E0F15000401040F7
:10096000E1F735C18C2F0E94E00336C18C2F8695AC
:100970008695837019F0813061F02EC1112321F02A
:100980008D2F9C2F937002C080E090E00E94DD16B6
:100990002BC1112321F08D2F9C2F937002C080E07A
:1009A00090E00E94F31620C18D2F112319F00E94B0
:1009B000501202C00E94AB120E94221315C18C2F4C
:1009C000837009F047C011110BC12D2F2295269578
:1009D0002770220F220F6D2F6F70862F90E0A0E0FE
:1009E000B0E0022E04C0880F991FAA1FBB1F0A94F3
:1009F000D2F7D4FF10C04FE050E060E070E004C0D8
:100A0000440F551F661F771F2A95D2F740955095C2
:100A10006095709503C040E050E0BA01C695C69558
:100A2000C3708A019B01082B192B2A2B3B2BC90170
:100A3000B801C23049F058F4C13019F00E94E806FC
:100A4000CFC00E94D606CCC00E94FA06C9C00E9440
:100A5000D406C6C0112319F08C2F817001C0869571
:100A6000882309F4BDC02D2F229526952770220FCB
:100A7000220F6D2F6F70862F90E0A0E0B0E0022E65
:100A800004C0880F991FAA1FBB1F0A94D2F7D4FF76
:100A900010C04FE050E060E070E004C0440F551F0C
:100AA000661F771F2A95D2F74095509560957095EF
:100AB00003C040E050E0BA01C695C695C3708A01F4
:100AC0009B01082B192B2A2B3B2BC901B801C230E3
:100AD00049F058F4C13019F00E94AD0781C00E945E
:100AE0009B077EC00E94BF077BC00E940E0778C094
:100AF000CF70112339F08C2F0E9434078D2F0E9464
:100B0000D9036EC08D2F0E94E0038C2F0E945507E1
:100B100067C0D23F21F128F4D03F41F0D13FC1F06E
:100B200043C0D33F19F1D43F79F03EC0112341F0C7
:100B3000053008F051C08C2F8F710E947A074CC08D
:100B4000063008F049C0F7CF8091720282FF18C0CA
:100B5000112339F08C2F8F710E9434073DC011236F
:100B6000C9F38C2F8F710E94550736C0112329F0CD
:100B70008C2F8F710E941F072FC00E941A072CC054
:100B8000112349F0CF718C2F0E94340763E08C2F22
:100B90000E94580C21C081E00E94730C0230E0F0EA
:100BA00082E00E94730C18C0112331F0002391F2EF
:100BB0008D2F0E94A70210C0002399F2D93349F467
:100BC0001FEF27EE33E0115020403040E1F700C026
:100BD00000008D2F0E94510388EF8C0D843020F48B
:100BE0000E94A9160E943C02DD20C9F00E94C60B9B
:100BF00080FD15C0F70112820E94C00B0E943407CD
:100C0000C7010E9430060E94C00BDF91CF911F9157
:100C10000F91FF90EF90DF90CF900C945507DF91EC
:100C2000CF911F910F91FF90EF90DF90CF9008959B
:100C30000F931F93CF93DF93EC01688179818A81B1
:100C40000E9478088C010E94D1070E94C206B80158
:100C5000CE010E94E703DF91CF911F910F9108957C
:100C6000CF93DF93EC01988189812B813C81232BE9
:100C700031F08F3F31F481E09F3F19F403C081E0F0
:100C800001C080E080FD1DC0CE010E94DA0181110B
:100C900010C00E94CA0B8823A1F08A81882389F0A2
:100CA0008091720282FD0DC082E0DF91CF910C94A1
:100CB000730CCE010E941806CE01DF91CF910C94E7
:100CC000BB01DF91CF91089580E090E00E94DD1696
:100CD00080E090E00E94F3160E94F10B0E94130C3A
:100CE0000E9453140C9422138091020190910301ED
:100CF0000E94B5170C9464060E94E10B0C947406D4
:100D000092959F70963079F010F4925001C09A50ED
:100D1000923068F4803F69F018F4883E40F409C0CE
:100D2000843F29F406C0883E20F0813F11F080E026
:100D3000089581E00895FC01808191810E946D08F1
:100D40000E9480060895CF93DF9300D000D01F92B9
:100D5000CDB7DEB70F900F900F900F900F90DF91EF
:100D6000CF910895CF93DF9300D000D000D0CDB7BE
:100D7000DEB726960FB6F894DEBF0FBECDBFDF916B
:100D8000CF910895089508950C94C3060C94C40659
:100D90000E94C6066093A2017093A3018093A401F0
:100DA0009093A5010C9464060C94C8060F931F93AE
:100DB0000091A2011091A3012091A4013091A501FD
:100DC000602B712B822B932B1F910F910C94C806D3
:100DD0000F931F930091A2011091A3012091A401F0
:100DE0003091A50160237123822393231F910F91DA
:100DF0000C94C8060F931F930091A2011091A301B8
:100E00002091A4013091A5016027712782279327A3
:100E10001F910F910C94C8060C94C3060E940C07F6
:100E200060939E0170939F018093A0019093A10114
:100E30000C94640660E070E0CB010C940E070F93F5
:100E40001F9341E050E060E070E08A019B0104C024
:100E5000000F111F221F331F8A95D2F7C901B80155
:100E60001F910F910C940E070F931F9341E050E0D8
:100E700060E070E004C0440F551F661F771F8A951D
:100E8000D2F780919E0190919F01A091A001B09115
:100E9000A1018A019B01082B192B2A2B3B2BC9018D
:100EA000B8011F910F910C940E070F931F9341E00F
:100EB00050E060E070E004C0440F551F661F771FCC
:100EC0008A95D2F7409550956095709580919E01D6
:100ED00090919F01A091A001B091A1018A019B0175
:100EE000082319232A233B23C901B8011F910F911D
:100EF0000C940E070F931F9341E050E060E070E008
:100F000004C0440F551F661F771F8A95D2F7809142
:100F10009E0190919F01A091A001B091A1018A0131
:100F20009B01082719272A273B27C901B8011F91D0
:100F30000F910C940E070F931F9300919E01109137
:100F40009F012091A0013091A101602B712B822B78
:100F5000932B1F910F910C940E070F931F930091E9
:100F60009E0110919F012091A0013091A101602369
:100F70007123822393231F910F910C940E070F93DB
:100F80001F9300919E0110919F012091A00130912B
:100F9000A10160277127822793271F910F910C943D
:100FA0000E07089524E0929F900D1124890FE82FD9
:100FB000E695E695E695877051E001C0550F8A9554
:100FC000EAF785E0E89FF0011124E657FE4F20E0A4
:100FD00030E070E04081CB01022E02C096958795EB
:100FE0000A94E2F781708195842785238427819371
:100FF0002F5F3F4F2530310569F7089524E0929F18
:10100000900D1124890F682F669566956695982F27
:10101000977085E0689FB001112440E050E080E0C7
:10102000FB01E40FF51FE657FE4F208130E0092E4B
:1010300002C0369527950A94E2F721703327042ED3
:1010400001C0220F0A94EAF7822B4F5F5F4F4530B1
:10105000510531F70895BF92CF92DF92EF92FF9240
:101060000F931F93CF93DF938C01C0909E01D0907C
:101070009F01E090A001F090A1018091A2019091C8
:10108000A301A091A401B091A501C82AD92AEA2AF6
:10109000FB2ACFE1D0E0D701C6010C2E04C0B695E3
:1010A000A795979587950A94D2F780FD04C021975C
:1010B00090F7B12C07C0BC2EB8018C2F0E945F0F97
:1010C0000197A9F38B2DDF91CF911F910F91FF9085
:1010D000EF90DF90CF90BF900895CF93DF93EC0116
:1010E0000E942B08BE010E945F0FDF91CF910895EF
:1010F0001F93CF93DF93EB0190918901992321F006
:10110000CB010E946D0813C0882349F0CB010E94D7
:101110002B08182F682FCE010E94D20704C0CB01E4
:101120000E94FE07182FBE01812F0E945F0FDF91E2
:10113000CF911F9108951F93CF93DF93C091A60184
:1011400016E08091A701C81799F0D0E01C9FF0012C
:101150001D9FF00D1124E855FE4F408151816281A1
:101160007381848195810E94B2062196C770E9CF70
:10117000DF91CF911F9108954091D8015091D901ED
:101180006091DA017091DB018091DC019091DD01C9
:101190000C94B206EF92FF920F931F93CF93DF93BD
:1011A0008091DD0182958F7009F065C08091DA0130
:1011B000882309F460C08091A601F090A7011091E6
:1011C000D8010091D9016091DB017091DC0191E0BF
:1011D0001F3F09F090E0C0910001D0910101292F3B
:1011E00096E0E92E8F1509F446C06115710521F0CE
:1011F0000F3F21F030E003C031E001C0322F90E01A
:1012000030FD36C0E89EF001E99EF00D1124DF01AB
:10121000A855BE4F11963C911197301329C03C91AF
:10122000311326C012963C911297311121C01396AA
:101230004D915C911497461B570B4C175D07C0F4FA
:101240008091DD018F7080618093DD01E355FE4F59
:1012500080818F708061808388ED91E00E943006EC
:10126000DF91CF911F910F91FF90EF900C949B080D
:1012700001968770B7CFDF91CF911F910F91FF90AB
:10128000EF9008959F92AF92BF92CF92DF92EF922C
:10129000FF920F931F93CF93DF93CDB7DEB7619784
:1012A0000FB6F894DEBF0FBECDBF8C0185E0F8010C
:1012B000DE011D9601900D928A95E1F7D8011296F4
:1012C000EC909091D801E091D9012091DB0130910F
:1012D000DC012115310531F0EF3F31F481E09F3F12
:1012E00019F403C081E001C080E0B82FB1709B2EDB
:1012F00080FD47C1D8014C9111965C9111971396CE
:10130000AD90BC90149788EDC82E81E0D82EF09057
:10131000DA01B501621B730B2091000130910101CC
:10132000FF2009F4D9C08091DD016217730708F02E
:1013300095C0282F207F09F052C05E1313C04913B7
:1013400011C0FE2CE1100EC08F7080618093DD0112
:101350000E94BC08C6010E9430068091DD01F801A0
:1013600085834DC1AB2831F05F3F31F481E04F3FC1
:1013700019F403C081E001C080E080FD03C081E07A
:101380008E2502C080E090E0F82FF170FF2E80FFE4
:101390001CC08091A6012091A70136E0821709F4B4
:1013A0000BC190E0389FF001399FF00D1124E855F2
:1013B000FE4F6181561306C06081461303C06281EF
:1013C000E61203C001968770E9CFFE2CEE2009F4E7
:1013D00016C18091DD0181608093DD0154C05E13F0
:1013E00006C0491304C0E11002C0F80199C0C80149
:1013F0000E949B06882361F1EE2051F12091DD01CE
:10140000822F82958F7090E0029774F08091D801BE
:101410009091D90198878F831986BB86AA862C87DD
:10142000CE0107960E94300686E0F801A8EDB1E0F3
:1014300001900D928A95E1F70E94CA080E94BC08AB
:101440000AC05E1711F1C8010E949B0681112CC0D1
:10145000C8010E943006FF24F394D1C0282F207FBA
:1014600081F77A2DB98AA88A6E2D89890E94A306F0
:1014700088ED91E00E94300686E0D6011D928A95A3
:10148000E9F70E94BC08F12CBAC04913DCCFE11087
:10149000DACFF8018583C8010E94300686E0D601C4
:1014A0001D928A95E9F7ABC0EE2091F22091DD0103
:1014B000822F82958F7090E002970CF4B5CF8091C7
:1014C000D8019091D9019A8389831B82BD82AC8215
:1014D0002E83CE010196A6CF6217730708F044C091
:1014E000FE2CEE2009F4B4CF5E1330C049132EC099
:1014F0002091DD0120FD21C0822F82958F70482F21
:1015000050E041155105C9F0F80125834F305105D0
:1015100041F08F5F982F9295907F822F8F70892B4B
:101520008583C8010E94300686E0F801A8EDB1E08D
:1015300001900D928A95E1F73CC086E0F801A8ED94
:10154000B1E001900D928A95E1F759C0C8010E945F
:101550009B06811169CF8091DD0181608093DD015F
:10156000C8010E9430064BC07A2DB98AA88A6E2D18
:1015700089890E94A30686E0D6011D928A95E9F723
:1015800018C0EE2009F464CFC8010E949B06F82E13
:10159000882309F45DCF86E0F801A8EDB1E0019061
:1015A0000D928A95E1F788ED91E00E94A1020E94D8
:1015B000CA080E94BC0823C04D875E878D859E8522
:1015C0000E946D08292F22952F70223028F49F70D9
:1015D00039F0811105C00BC0243028F49F7049F404
:1015E000805E883020F0C8010E9430069F2CF92CC4
:1015F00006C0D80115969C91907F91F7F8CF8F2D5A
:1016000061960FB6F894DEBF0FBECDBFDF91CF91CC
:101610001F910F91FF90EF90DF90CF90BF90AF9010
:101620009F9008951F93CF93DF93CDB7DEB72C978C
:101630000FB6F894DEBF0FBECDBF4F8358876987C2
:101640007A878B879C87CE0107960E944209882360
:10165000D1F09F8188852A853B85232B31F08F3FF0
:1016600031F481E09F3F19F403C081E001C080E0C4
:1016700080FD47C04F81588569857A858B859C851B
:101680000E94B2063EC086E0FE013796DE0111964A
:1016900001900D928A95E1F7FF81E8856A857B8547
:1016A0006115710531F0EF3F31F481E0FF3F19F42E
:1016B00003C081E001C080E080FD23C02091A7012C
:1016C00030E0C9010196877099274091A60150E04A
:1016D00084179507F1F1F983EA837D836C8396E0A3
:1016E000929FD001939FB00D1124A855BE4FFE01CB
:1016F000319601900D929A95E1F78093A7010E948F
:101700009B0816E08091A6019091A701891771F1BD
:10171000189FC001112488559E4F0E9442098823BA
:1017200029F1E091A6011E9FF0011124E855FE4F1A
:101730004081518162817381848195810E94B206CA
:101740008091A60190E00196877099278093A60169
:10175000D9CF0E947C061092A7011092A601E8ED55
:10176000F1E086E0DF011D928A95E9F72C960FB62D
:10177000F894DEBF0FBECDBFDF91CF911F910895CA
:101780008091FE0185958595859508958091FE014E
:10179000877008959091FE01977081E009F480E0D0
:1017A000089580912102089590912102892B8093C0
:1017B000210208958095909121028923809321022E
:1017C000089510922102089590912002892B809310
:1017D0002002089580959091200289238093200211
:1017E00008951092200208958091FF0108950895B0
:1017F0000C94F70B0C94F80B9091720292FD08C0B8
:101800009091FF01981721F08093FF010C94FA0B3F
:1018100008958091FF01882329F01092FF0180E054
:101820000C94FA0B0895CF93DF93E0910201F091AD
:101830000301809121028083E0910201F091030174
:10184000908180912002892B80838091FF018823E1
:1018500081F0E0910201F09103019081892B808356
:1018600080910201909103010E94091781110E9449
:10187000090CC0910201D091030140E250E06EEDED
:1018800071E0CE010E94CF1F892B69F080E2FE013A
:10189000AEEDB1E001900D928A95E1F7CE01DF91B6
:1018A000CF910C94B516DF91CF9108950C94F70B5E
:1018B0009091720292FD10C098E0899F90011124CE
:1018C000262B2093FE010E9434078091FE0185950E
:1018D000859585950C94560C0C9434071092FE0156
:1018E00080E00C94560C2091FE0180958223809319
:1018F000FE01982F977099F430E0482F082E000CC5
:10190000550B2417350759F09091720292FD07C0CC
:101910008595859585950E9455070C946E0C0895C4
:101920009091720292FB222720F9281769F080FB20
:1019300092F99093720280917102909172020E94CA
:10194000DE0C82E00C94730C08958091720282FB8D
:10195000882780F991E089270C94900C81E00C9401
:10196000900C80E00C94900C6FEF7FEF80E090E0A3
:101970000C94082080E090E00E94E41F21E0893E62
:101980009E4F09F020E0822F089582E090E00C94B1
:10199000DC1F83E090E00C94DC1FCF9384E090E0A8
:1019A0000E94DC1FC82F82E290E00E94DC1F2C2FD7
:1019B00030E0A901582BCA01CF910895CF93C92FC8
:1019C000682F84E090E00E94EA1F6C2F82E290E092
:1019D000CF910C94EA1FAB01BC018FE090E00C9416
:1019E000FC1FAB01BC0183E190E00C94FC1F60E0A4
:1019F00070E0CB010C94F10C60E070E0CB010E9430
:101A0000EB0C0C94F70C69EE7EEF80E090E00E9406
:101A1000082060E082E090E00E94EA1F60E083E03E
:101A200090E00E94EA1F1092A2011092A30110926E
:101A3000A4011092A50160E084E090E00E94EA1FFA
:101A400060E082E290E00E94EA1F60E085E090E0C2
:101A50000E94EA1F60E086E090E00E94EA1F6FEFBC
:101A600087E090E00E94EA1F40E050E0BA0188E081
:101A700090E00E94FC1F60E08DE090E00E94EA1F71
:101A800040E050E0BA0188E190E00E94FC1F60E075
:101A900087E190E00E94EA1F40E050E0BA018CE14B
:101AA00090E00E94FC1F60E070E080E290E00E9405
:101AB000082040E050E0BA0188E190E00E94FC1F5D
:101AC0000C94FC0C0C94030D682F8EE090E00C94A9
:101AD000EA1F0E946E1860932B0270932C02809371
:101AE0002D0290932E026093270270932802809318
:101AF000290290932A02089585B7806885BF85B72B
:101B0000806885BF089581E008950C94830D089541
:101B10000C94870D0C94870D0C948A0D0C94870DF2
:101B20000C948E0D0C94870D0E947C0D8BE390E13C
:101B30000E949F160E94920D0C94900D0E94880D99
:101B40000C94870D0E9455100C943B020E9459186A
:101B50000E942C110E94A20D0C948C0D8F929F92CA
:101B6000AF92BF92CF92DF92EF92FF920F931F93AB
:101B7000CF93DF93CDB7DEB72A970FB6F894DEBFC9
:101B80000FBECDBF0E944111982E81110E94690D98
:101B900082E2A82E82E0B82E00E010E0802E802F96
:101BA0000E947910D82EF501C1905F01C826B1F4CA
:101BB0000F5F1F4F0530110589F78FEF89838A83E7
:101BC0001B820E9462188160782F9D838C834981DB
:101BD0005A816B818D810E9457022FC080912F0204
:101BE00081FD0E947F10E12CFF24F3948C2D8F2126
:101BF000F1F00E94850D882399F0EE828F82DF201C
:101C000081E009F480E088870E9462188160782F63
:101C10009A8789874E815F8168858A850E945702ED
:101C2000F801EE5DFD4F8081F826F08206C0E39456
:101C3000FF0CF5E0EF12DACFBBCF81E0911001C0CD
:101C400080E02A960FB6F894DEBF0FBECDBFDF91BD
:101C5000CF911F910F91FF90EF90DF90CF90BF90A9
:101C6000AF909F908F9008950E94AE0D0E944013F8
:101C70000C944C02CF93DF930E94640FEC0181150A
:101C800021E5920708F045C0811530E5930708F07B
:101C900094C0883E910528F5803E910508F0F8C073
:101CA000883A910570F4853A910508F07CC081303E
:101CB000910509F475C008F4E8C0049708F0E8C07D
:101CC000E4C08F3B910508F0E0C0C85AD0E0CC0FCB
:101CD000DD1FC65BDE4F0990D881C02DCE01946414
:101CE000D8C0811540E2940758F4811551E095075A
:101CF00008F0CEC08D3E910508F4C7C09065C9C0FC
:101D0000C11580E4D80708F4C0C0DF70CE01906A26
:101D1000C0C0811525E59207A8F4811534E5930725
:101D200008F095C0811543E5940708F07BC0811544
:101D300052E5950708F061C0D82FCC27CE01816FFE
:101D4000906AA7C0C11589E5D807A0F4C11528E598
:101D5000D20708F082C0C11536E5D30708F095C058
:101D60008C2F0E94F80F8F7190E0D82FCC27CE01D6
:101D700090628FC0C1154AE5D40708F474C0CE0143
:101D800090568115904208F080C08D2F8F710E946F
:101D9000F80FDD27D0628F71AE01582BCA0179C0D0
:101DA00081E090E076C0C55AD0E0C858DE4F888107
:101DB000C82FD0E0CE0190646CC074E096958795F2
:101DC0007A95E1F7282F23703C2F337081E090E063
:101DD00002C0880F991F3A95E2F79C68AC01522B1C
:101DE0009A019C2F9F709695969550E2959FE001E1
:101DF0001124C9018C2B9D2B4CC08370992721E0A5
:101E000030E002C0220F331F8A95E2F79C2F96958F
:101E1000969580E2989FE0011124C22BD32BCE012E
:101E20009C6837C08370992721E030E002C0220F00
:101E3000331F8A95E2F79C2F9695969540E2949FE2
:101E4000E0011124C22BD32BCE019A6822C0D82FD7
:101E5000CC27CE01846F906A1CC0DC2FCC27CE012A
:101E6000806F906A16C08C2F8F700E94F80F94E0DC
:101E7000D695C7959A95E1F7CF70D0E0DC2FCC27A7
:101E8000D0699E01282BC90104C080E090E001C008
:101E9000CE01DF91CF91089529E1829FC0011124E5
:101EA000FC0125E0729FE00DF11D1124E60FF11DEC
:101EB000EE0FFF1FE852FF4F8591949108950E9405
:101EC0004C0F0E943A0E08958238910569F1B0F4E2
:101ED0008133910509F46DC048F48932910509F404
:101EE00063C08A32910509F469C00895853391056C
:101EF00009F455C089339105B9F00895833E9105E1
:101F000069F138F4803E9105B1F0823E910509F106
:101F10000895863E9105A9F1873E9105B9F1843E69
:101F2000910509F064C023C02091710220FD4FC0CB
:101F300021FD4DC008958091710280FD44C08091C3
:101F4000720280FF44C08091710284FD42C083EE22
:101F50004DC08091710282FF38C0F5CF809171022F
:101F600082FD33C08091720280FD31C0ECCF809140
:101F7000720281FF32C08091710284FD2AC087EE17
:101F800035C08091710283FF26C0F5CF8091710228
:101F900083FD21C08091720281FD1FC0ECCF809132
:101FA000710285FD1CC01DC08091710285FD19C0A4
:101FB00016C08091710286FD16C017C08091710213
:101FC00086FD13C010C089E311C082EE0FC080EE01
:101FD0000DC080E00BC086EE09C084EE07C089E228
:101FE00005C085E303C08AE201C081E390E0089563
:101FF0009091710292FF0DC0282F2871283019F49A
:10200000877F846006C0282F2471243011F48B7FD1
:10201000886093FF0DC0282F2871283119F4877E1E
:10202000846106C0282F2471243111F48B7E8861CD
:102030002091720220FF0DC0382F3871383019F40A
:10204000877F816006C0382F3171313011F48E7F67
:10205000886021FF0DC0282F2871283119F4877E50
:10206000816106C0282F2171213111F48E7E886193
:1020700094FD877E089580E008950C94B40C0E942E
:1020800041118FE39CE90197F1F700C000000E9425
:10209000411180E00E94791080FF04C00E943D1031
:1020A0000C94AF1808950C943F100E94BA0C811143
:1020B00002C00E94620D0E94C50C80932F020E94F4
:1020C000CD0C90937202809371020E9453100E9473
:1020D000C90C682F70E080E090E00E94D406609107
:1020E0009E0170919F018091A0019091A1010C949B
:1020F0000C07E82FF0E0E858FD4F8081089508951F
:1021000080EA8A95F1F7089500C008950C94801034
:1021100008950C9488100C9489100C9488100C94D9
:102120008D10F894E82FE295EF70F0E031A1282FA0
:102130002F7081E090E001C0880F2A95EAF7982F70
:102140009095932391A392A1892B82A378940895CB
:102150000F931F93CF93DF93C0E8D1E089918F3F16
:1021600011F00E94911081E0C538D807B9F7CBE78C
:10217000D1E000E811E089918F3F11F00E949110A9
:102180000C171D07C1F7DF91CF911F910F91089593
:10219000CF92DF92EF92FF920F931F93CF93DF9333
:1021A0008C01C62FD0E0CE0180589E4F7C01FC01EF
:1021B00090819F3F09F447C0D62EF894E92FE2950D
:1021C000EF70F0E081A19F7021E030E001C0220FAC
:1021D0009A95EAF7822B81A382A12095282322A336
:1021E00078940E948410EBE7F1E040E851E031E0A0
:1021F000C12C21912F3F89F0A22FA295AF70B0E0A2
:1022000090968C9190E02F7002C0959587952A95B5
:10221000E2F780FD02C0832F01C080E0C82A330F9F
:102220004E175F0731F7F70180818F3F11F00E9451
:10223000911061E0C11001C060E08D2D0E948610F8
:10224000C00FD11FC882DF91CF911F910F91FF90D6
:10225000EF90DF90CF9008950E94A81085E0E8E706
:10226000F2E0DF01982F1D929A95E9F7E3E7F2E09B
:10227000DF011D928A95E9F785E00E9488110C9490
:10228000C601FF920F931F93CF93DF9300D000D02E
:102290001F92CDB7DEB78E010F5F1F4F85E0F801AB
:1022A00011928A95E9F7F12C6F2DC8010E94C81090
:1022B000F394F5E0FF12F8CF45E050E0B80183E772
:1022C00092E00E94CF1FFF24F394009709F4F12CB1
:1022D000892B41F085E0F801A3E7B2E001900D926F
:1022E0008A95E1F72F2D45E068E772E083E792E0F9
:1022F0000E9489110E94C8018F2D0F900F900F909E
:102300000F900F90DF91CF911F910F91FF90089543
:102310000895FF920F931F93CF93DF938C01F62EB6
:10232000D72FC42F222349F081E0809332020E94EC
:102330006218909331028093300280913202882398
:10234000C1F080913002909131020E947A18059775
:1023500080F0EF2DFD2FD8014C2F50E0CD01801BD8
:10236000910B841795071CF48D918193F7CF1092F0
:102370003202DF91CF911F910F91FF9008950E943B
:10238000671A0E94A60D0C94731A0E94771A0E9475
:10239000340E0C94911A0E9400180E944E1A0E944A
:1023A000940D0E94BF110E94C5110E949E0DFBCF8B
:1023B0008091390280FF06C06091090170E0660FCC
:1023C000771F26C081FF04C06091090184E005C029
:1023D00082FF07C06091090188E0689FB001112465
:1023E00017C0909138029923D1F060910801961797
:1023F00088F72091090188E0289F90011124929F7D
:10240000A001939F500D112470E0CA010E94A11FEA
:102410006038710540F46115710519F406C068E073
:1024200070E0862F08958FE7089581E008958091E8
:10243000390280FF08C06091050170E075956795CD
:102440007595679521C081FF06C06091050170E018
:102450007595679519C082FF04C06091050170E011
:1024600010C090913702992399F06091040196175A
:10247000A0F780910501899FC001112470E00E949E
:10248000A11F6038710540F46115710519F406C08B
:1024900061E070E0862F08958FE7089581E0089548
:1024A0008D3E21F40E94D811819504C08E3E29F4FE
:1024B0000E94D81180933D0208958F3E21F40E941E
:1024C000D811819504C0803F29F40E94D8118093CF
:1024D0003C020895893F19F40E94171205C08A3FF3
:1024E00031F40E941712819580933E0208958B3F2C
:1024F00021F40E941712819504C08C3F29F40E9498
:10250000171280933F0208959FE0980F983078F457
:1025100021E030E0A90102C0440F551F9A95E2F76F
:10252000CA0190913B02892B80933B0208958D3F15
:1025300021F48091390281600BC08E3F21F480919B
:102540003902826005C08F3F29F48091390284608E
:102550008093390208958D3E39F490913D0297FFA2
:1025600035C010923D0259C08E3E29F490913D0233
:102570001916BCF32BC090913C028F3E29F497FFB3
:1025800025C010923C0249C0803F19F41916CCF3C3
:102590001DC090913E02893F29F41916BCF4109297
:1025A0003E023BC08A3F19F497FF10C0F8CF8B3F23
:1025B00039F490913F0297FF09C010923F022DC05D
:1025C0008C3F21F490913F021916BCF39FE0980FC5
:1025D000983080F421E030E0A90102C0440F551F7B
:1025E0009A95E2F7CA01809590913B0289238093E6
:1025F0003B0213C08D3F21F4809139028E7F0BC0C6
:102600008E3F21F4809139028D7F05C08F3F29F4E0
:10261000809139028B7F8093390280913C02811135
:1026200006C080913D02811102C010923802809153
:102630003E02811106C080913F02811102C01092BA
:10264000370208950E94621820913C02211104C0B3
:1026500020913D02222321F090933602809335028F
:1026600020913E02211104C020913F02222321F03B
:1026700090933402809333028AE392E00C94CF1655
:10268000EF92FF920F931F93CF93DF9300D000D070
:1026900000D0CDB7DEB786E0EAE3F2E0DE011196C6
:1026A00001900D928A95E1F7E0903C02F0903D0296
:1026B00000913E0210913F0210923C0210923D02A6
:1026C00010923E0210923F02E11003C0FF2009F475
:1026D0005DC080913502909136020E947A18AC015B
:1026E00090913802992339F020910A0130E02417A3
:1026F000350758F04BC020910B018AE0289F9001CC
:1027000011242417350718F041C09F3F19F09F5F2F
:1027100090933802EE2061F00E94D8111E1414F03C
:102720009FEF01C091E0989F902D112490933C025F
:10273000FF2061F00E94D8111F1414F09FEF01C018
:1027400091E0989F902D112490933D0230913C028E
:102750003323E1F020913D022223C1F045EB340305
:10276000C0011124992319F090933C0203C081E029
:1027700080933C0235EB2303C0011124992319F007
:1027800090933D0203C081E080933D02011103C09C
:10279000112309F45DC080913302909134020E94AC
:1027A0007A18AC0190913702992339F020910601F3
:1027B00030E02417350758F04BC0209107018AE01C
:1027C000289F900111242417350718F041C09F3F1E
:1027D00019F09F5F90933702002361F00E94171257
:1027E000101614F09FEF01C091E0989F902D1124D6
:1027F00090933E02112361F00E941712111614F0FB
:102800009FEF01C091E0989F902D112490933F027B
:1028100030913E023323E1F020913F022223C1F0A8
:1028200045EB3403C0011124992319F090933E0223
:1028300003C081E080933E0235EB2303C0011124E5
:10284000992319F090933F0203C081E080933F02E7
:1028500080913C0281110BC080913D02811107C023
:1028600080913E02811103C080913F0281110E943C
:102870002213EB82FC820D831E8386E0FE013196DB
:10288000AAE3B2E001900D928A95E1F726960FB681
:10289000F894DEBF0FBECDBFDF91CF911F910F9196
:1028A000FF90EF900895EAE3F2E086E0DF011D92E9
:1028B0008A95E9F710923802109237021092390285
:1028C0000895CF93DF93EC01FB018281882309F403
:1028D0003CC1C430FDE5DF0760F4CB3F9CE5D90780
:1028E00088F49E0122503C452431310508F02EC168
:1028F00009C0C236EDE5DE0729F0C63AFDE5DF077F
:1029000009F024C10E94CD0C909372028093710251
:10291000C1318CE5D80709F4C6C008F042C0C930FF
:10292000ECE5DE0709F49BC000F5C5308CE5D8075F
:1029300009F485C078F4C330ECE5DE0709F478C00B
:1029400008F07AC0C230DC4509F0F5C08091710210
:102950008160EFC0C7309CE5D90709F478C008F062
:102960007AC0809171028061E4C0CD30FCE5DF0760
:1029700009F487C058F4CB309CE5D90709F479C035
:1029800008F07BC08091710288606FC0CF30FCE599
:10299000DF0709F480C008F082C080917102877F50
:1029A000C8C0CE3F9CE5D90709F471C000F5C53118
:1029B000FCE5DF0709F485C068F4C3319CE5D9075D
:1029C00009F475C008F095C00E947C0680917102E0
:1029D0008F77AFC0CC3FFCE5DF07A9F108F054C00A
:1029E000CB3FDC4509F0A7C08091720240C0C230E5
:1029F000EDE5DE0709F489C058F4C1158DE5D80767
:102A000009F45AC008F069C08091720282602FC038
:102A1000C236EDE5DE0709F47CC0C63AFDE5DF0706
:102A200009F481C0C330DD4509F085C080E06EC087
:102A30008091710282607DC08091710216C0809188
:102A40007102886076C08091720282604FC080916E
:102A5000710280626EC08091710280646AC00E94BF
:102A60007C0680917102806864C0846062C081606D
:102A70003DC0809171028E7F5CC0809171028D7F1C
:102A800058C08091710216C08091720218C0809166
:102A900072028D7F2BC0809171028F7E4AC080911F
:102AA00071028F7D46C0809171028F7B42C0809100
:102AB0007102877F8B7F3DC0809172028D7F8E7FF8
:102AC00015C08091710282FB222720F991E09227A4
:102AD00090FB82F990FB83F92CC080917202982FB1
:102AE000909591708E7F892B90FB81F98093720273
:102AF00022C00E947C068091710287FB222720F968
:102B000091E0922790FB87F914C081E00E94640D48
:102B100012C08091710284FB222720F991E0922754
:102B200090FB84F906C080917102982F909590FBDC
:102B300080F98093710280917102909172020E94DB
:102B4000DE0C0E947C0680E001C081E0DF91CF9125
:102B50000895CF93DF9386319C4541F5EB010E94A8
:102B6000D10B982F8A812091020130910301882393
:102B700079F09A7A81E009F480E080934002911123
:102B800002C069E201C065E3C9010E949F170AC043
:102B900080914002811102C069E201C065E3C90170
:102BA0000E94AA170E94130C80E001C081E0DF910F
:102BB000CF9108950F931F93CF93DF93C42FD22FFC
:102BC000FC0182818823C9F0409343020E9462186D
:102BD000909342028093410280E28C0F883008F08B
:102BE00057C0C77081E001C0880FCA95EAF7DF912E
:102BF000CF911F910F910C94D903809143024813F8
:102C000030C080914102909142020E947A18883C23
:102C1000910538F510E21D0FCD17B9F080E28C0F49
:102C2000883040F4C77081E001C0880FCA95EAF788
:102C30000E94E003183028F581E09D2F977001C0B5
:102C4000880F9A95EAF70E94D903802F0E94D0033B
:102C50001830F0F4D77081E001C0880FDA95EAF7F8
:102C60000AC080E28C0F883098F4C77081E001C000
:102C7000880FCA95EAF7DF91CF911F910F910C94BD
:102C8000E003802FDF91CF911F910F910C94D0031F
:102C9000DF91CF911F910F9108950F939C01CB016C
:102CA000243F4CE5340731F188F4293DFCE53F072A
:102CB000D9F02A3D4CE5340779F1283D3C45A9F58A
:102CC00006E221EE41EE68ED7CE52BC0263FFCE5F7
:102CD0003F07E1F0A8F0273F3C4539F507E225EE34
:102CE00046EE67EF7CE51DC007E225EE45EE69ED97
:102CF0007CE517C006E221EE40EE64EF7CE511C0F2
:102D000007E225EE44EE65EF7CE50BC006E221EE1E
:102D100042EE66EF7CE505C008E221E045EE6AED93
:102D20007CE50E94DA1580E008C0FC0182818823DE
:102D300019F01092430201C081E00F910895909321
:102D400087018093860108959093490280934802F9
:102D50000895E0914802F0914902309721F00190E6
:102D6000F081E02D099480E00895E0914802F0910F
:102D70004902309799F020911801222359F02091AF
:102D8000710227FF07C0DC012C9111962C9311973B
:102D900026E02C930280F381E02D09940895E091C0
:102DA0004802F0914902309739F022E0DC012C937F
:102DB0000480F581E02D0994089520914602309118
:102DC00047022817390771F0909347028093460213
:102DD000E0914802F0914902309721F00680F78196
:102DE000E02D09940895209144023091450228175E
:102DF000390771F09093450280934402E0914802B4
:102E0000F0914902309721F00084F185E02D09947A
:102E10000895FC01329680911801882331F0809149
:102E2000710287FF02C09EE101C096E080E09150F0
:102E300028F021912223D9F38F5FF9CF08956623DB
:102E400051F1209118012223E9F02091710227FF0E
:102E500019C0462F4695469546954E31E0F4677069
:102E600021E030E002C0220F331F6A95E2F7FC0137
:102E7000E40FF11D828190E02823392381E0232B88
:102E800069F409C0FC01329608962191621729F075
:102E9000E817F907D1F780E0089581E008959C01D3
:102EA000FC0132969FEF80E04191461789F09F3FE9
:102EB00019F4411101C0982F8F5F8630A9F79F3F09
:102EC00039F0F901E90FF11D97FDFA956283089534
:102ED00008959C012A5F3F4FFC014281461301C0C7
:102EE0001282019682179307B9F70895262F269527
:102EF000269526952E3168F4FC01E20FF11D6770CE
:102F000021E030E001C0220F6A95EAF78281282B88
:102F100022830895262F2695269526952E3170F426
:102F2000FC01E20FF11D677021E030E001C0220FCB
:102F30006A95EAF7209582812823228308952091BB
:102F40001801222329F02091710227FD0C94761795
:102F50000C944F1720911801222329F0209171021F
:102F600027FD0C948A170C94691720911801FC0115
:102F70003296222331F08091710287FF02C08EE1E8
:102F800001C086E0DF011D928A95E9F70895089552
:102F90000C94C71783E080934A020C94C8178111E0
:102FA00002C081E001C082E080934A020C94C817FD
:102FB0000C94CF1781E080934A020C94C8170C94AC
:102FC000DA1708950C94E1170C94E2170C94E117AA
:102FD0000C94E1170C94E117CF930E94E8170E941C
:102FE00041110E94E617C0E08C2F0E9479108111D8
:102FF00004C0CF5FC530C1F701C081E0CF91089513
:1030000008951F920F920FB60F9211248F939F93E2
:10301000AF93BF9380914B02811113C080917D02C9
:1030200090917E02A0917F02B09180024196A11DF5
:10303000B11D80937D0290937E02A0937F02B09396
:103040008002BF91AF919F918F910F900FBE0F9013
:103050001F90189580918502843031F10E942C02D6
:1030600010924B0220E488E190E00FB6F894A89506
:10307000809360000FBE2093600083B7817F8460DF
:1030800083BF83B7816083BF7894889583B78E7F31
:1030900083BF0FB6F894A8958091600088618093F3
:1030A0006000109260000FBE08950E947C060C9490
:1030B000300282E084BD93E095BD9AEF97BD809386
:1030C0006E0008952FB7F89480917D0290917E0252
:1030D000A0917F02B09180022FBF08952FB7F8947E
:1030E00060917D0270917E0280917F0290918002BA
:1030F0002FBF08959C014FB7F89480917D02909165
:103100007E02A0917F02B09180024FBF821B930B81
:10311000089578941F920F920FB60F9211248F93F7
:103120009F93AF93BF9380917D0290917E02A09177
:103130007F02B09180020196A11DB11D80937D0296
:1031400090937E02A0937F02B0938002BF91AF91D3
:103150009F918F910F900FBE0F901F90189587E74A
:1031600097E790930108809300089AE088E10FB6F2
:10317000F894A895809360000FBE90936000FFCFF5
:1031800080916F020895089522E02093E9002FEFC7
:103190003091E800215035FD06C035ED3A95F1F744
:1031A00000002111F5CF2091E80025FF0BC040E081
:1031B00050E066E070E00E94031B8091E8008E778B
:1031C0008093E8000895CF93DF9320911801222384
:1031D00039F02091710227FF03C060E222E002C0B3
:1031E00068E021E02093E9002FEF3091E8002150C2
:1031F00035FD06C035ED3A95F1F700002111F5CF08
:103200002091E80025FF1DC0EC018091180181117B
:1032100005C040E050E068E070E003C070E040E0CE
:1032200050E0CE010E94031B8091E8008E778093CE
:10323000E80080E2FE01AFE4B2E001900D928A95D1
:10324000E1F7DF91CF91089580934C0270934E0285
:1032500060934D0280918502843001F582E0809375
:10326000E9008FEF9091E800815095FD06C095ED43
:103270009A95F1F700008111F5CF8091E80085FF64
:103280000DC040E050E063E070E08CE492E00E940A
:10329000031B8091E8008E778093E8000895BC01BD
:1032A00084E00C942419BC0183E00C9424198091CF
:1032B0008402811109C00E94941C0E94F11C80911B
:1032C000E20084608093E2000895109284020895E1
:1032D0000C94DF176091810281E0611101C080E0F0
:1032E0000C94CA179091850281E0943009F080E037
:1032F000609181020C94CF1742E061EC81E00E9462
:103300000D1C42E261EC82E00E940D1C909185024E
:1033100081E0943009F080E0609181020C94D8172C
:1033200080918702833009F461C030F4813071F0FC
:10333000823009F49AC008958A3009F486C08B302F
:1033400009F46CC0893009F0A8C020C080918602C1
:10335000813A09F0A2C08091E800877F8093E8005D
:1033600080918A0290918B02892B21F460E28FE494
:1033700092E003C060E080E090E070E00E944E1BAD
:103380008091E8008B778093E80008958091860211
:10339000813209F082C080918A0290918B0202975B
:1033A00008F07BC08091E800877F8093E8008091DF
:1033B000E80082FD05C0809185028111F8CF6DC0C3
:1033C0002091F3008091F20090E0922B029731F46B
:1033D0008091F100813011F0863021F48091F1006C
:1033E00080936F028091E8008B7753C080918602B2
:1033F000813A09F052C080918A0290918B02892B08
:1034000009F04BC08091E800877F8093E8008091AD
:10341000E80080FFFCCF8091180136C080918602C1
:103420008132D9F580918A0290918B02892BA9F57E
:103430008091E800877F8093E8000E94421C809181
:103440008802809318010C947C0680918602813258
:1034500021F58091E800877F8093E8000E94421C5C
:103460008091890280937002089580918602813A4A
:10347000A1F48091E800877F8093E8008091E800C4
:1034800080FFFCCF809170028093F1008091E80072
:103490008E778093E8000C94421C089584B7877F50
:1034A00084BF0FB6F894A8958091600088618093DE
:1034B0006000109260000FBE90E080E80FB6F894B4
:1034C00080936100909361000FBE0C94DA170E9404
:1034D000941C0E94F11CE2EEF0E080818460808305
:1034E00078940C94861F8CE091E00C94A416809143
:1034F00085028530A9F480918502853079F40E9497
:103500002A18809183028823B1F30E94EC17882344
:1035100091F30E94ED1A0E947C06EDCF0C94551891
:10352000089508950C94941A292F332723303105D8
:10353000C9F060F42130310581F02230310509F005
:1035400044C08BE390E026E631E043C021323105F0
:10355000E1F02232310549F138C082E190E021EA00
:1035600031E037C099278130910549F028F0029762
:1035700061F5ECE3F1E005C0E2E6F1E002C0E0E570
:10358000F1E0849190E09F0124C06115710541F044
:1035900061307105D1F489E090E021E931E019C092
:1035A00089E090E028E731E014C06115710541F031
:1035B0006130710551F486EB90E023EB31E009C0F6
:1035C00080E490E029E632E004C080E090E020E072
:1035D00030E0FA0131832083089580E189BD82E1E2
:1035E00089BD09B400FEFDCF8091D8008F7D809306
:1035F000D8008091E00082608093E0008091E0003C
:1036000081FDFCCF0895CF92DF92EF92FF920F934E
:103610001F93CF93DF93EC018B017A010E94611C11
:10362000811133C0E114F10439F0F70180819181F7
:10363000081B190BC80FD91FC12CD12C011511055E
:1036400019F18091E80085FD16C08091E8008E7721
:103650008093E800E114F10449F0F7018081918141
:10366000C80ED91ED182C08285E00FC00E94611CA5
:10367000882321F30AC089918093F1000150110938
:10368000FFEFCF1ADF0ADACF80E0DF91CF911F91F1
:103690000F91FF90EF90DF90CF90089520918C02D2
:1036A00030918D022617370748F06115710539F4FE
:1036B0002091E8002E772093E80001C0B901FC01B9
:1036C00020E06115710579F1809185028823F1F17F
:1036D0008530F1F18091E80083FD3CC08091E800E5
:1036E00082FD2EC08091E80080FFEBCF2091F30097
:1036F0008091F20090E0922B6115710551F08830B5
:10370000910538F421912093F100615071090196DF
:10371000F3CF21E0089709F020E08091E8008E7750
:103720008093E800CECF2111CFCF0AC080918502CF
:10373000882361F0853061F08091E80083FD0AC044
:103740008091E80082FFF2CF80E0089582E0089542
:1037500083E0089581E0089520918C0230918D02DC
:103760002617370748F06115710539F42091E800F4
:103770002E772093E80001C0B901FC0120E061151B
:10378000710591F180918502882309F440C085304C
:1037900009F43FC08091E80083FD3DC08091E800BE
:1037A00082FD2FC08091E80080FFE9CF2091F300D7
:1037B0008091F20090E0922B6115710559F08830EC
:1037C000910540F424912093F100319661507109E4
:1037D0000196F2CF21E0089709F020E08091E800FF
:1037E0008E778093E800CBCF2111CCCF0AC0809197
:1037F0008502882361F0853061F08091E80083FDC7
:103800000AC08091E80082FFF2CF80E0089582E054
:10381000089583E0089581E00895982F973068F522
:103820009093E900981739F07091EC002091ED0029
:103830005091F00003C0242F762F50E021FD02C0EC
:103840009F5FECCF3091EB003E7F3093EB003091E7
:10385000ED003D7F3093ED003091EB00316030930F
:10386000EB007093EC002093ED005093F00020915A
:10387000EE0027FDE5CF80E008958F708093E9008A
:1038800081E008958091860287FF11C08091E80051
:1038900082FD05C0809185028111F8CF11C0809111
:1038A000E8008B770BC080918502882349F08091D6
:1038B000E80080FFF8CF8091E8008E778093E800E1
:1038C00008952091E4003091E50095E64091EC00E8
:1038D000842F817040FF23C08091E80080FD1DC0CF
:1038E00080918502882399F0853099F08091EB00D2
:1038F00085FD11C04091E4005091E5002417350783
:1039000029F3915011F09A01E1CF84E0089582E00B
:10391000089583E0089581E0089580E0089540913E
:10392000E80042FFDDCF08950E94021D0E940A1D9B
:10393000E0EEF0E0808181608083E8EDF0E080815E
:103940008F77808319BCA7EDB0E08C918E7F8C932C
:1039500080818F7E80831092840208950F931F933D
:10396000CF93DF930E94021D0E940A1DC8EDD0E094
:1039700088818F77888388818068888388818F7D1C
:10398000888319BC109285021092810210928302E2
:103990001092820200EE10E0F80180818B7F80831C
:1039A00088818160888342E060E080E00E940D1C95
:1039B000E1EEF0E080818E7F8083E2EEF0E08081B6
:1039C00081608083808188608083F80180818E7F20
:1039D0008083888180618883DF91CF911F910F91CF
:1039E0000895E8EDF0E080818F7E8083E7EDF0E0E0
:1039F00080818160808384E082BF81E08093840243
:103A00000C94AE1CE8EDF0E080818E7F80831092F4
:103A1000E20008951092DA001092E10008951F92DA
:103A20000F920FB60F9211242F933F934F935F93F2
:103A30006F937F938F939F93AF93BF93EF93FF9376
:103A40008091E10082FF0BC08091E20082FF07C0FD
:103A50008091E1008B7F8093E1000E94851F80911F
:103A6000DA0080FF1FC08091D80080FF1BC08091CA
:103A7000DA008E7F8093DA008091D90080FF0DC03C
:103A800080E189BD82E189BD09B400FEFDCF81E0FE
:103A9000809385020E94571905C019BC10928502B7
:103AA0000E9465198091E10080FF19C08091E200B9
:103AB00080FF15C08091E2008E7F8093E2008091AC
:103AC000E20080618093E2008091D8008062809360
:103AD000D80019BC85E0809385020E946A19809104
:103AE000E10084FF30C08091E20084FF2CC080E1BF
:103AF00089BD82E189BD09B400FEFDCF8091D80067
:103B00008F7D8093D8008091E1008F7E8093E100CB
:103B10008091E2008F7E8093E2008091E2008160DC
:103B20008093E20080918102882311F084E007C035
:103B30008091E30087FD02C081E001C083E08093B3
:103B400085020E9472198091E10083FF29C0809153
:103B5000E20083FF25C08091E100877F8093E10030
:103B600082E080938502109281028091E1008E7F35
:103B70008093E1008091E2008E7F8093E20080914B
:103B8000E20080618093E20042E060E080E00E9419
:103B90000D1C8091F00088608093F0000E946819ED
:103BA000FF91EF91BF91AF919F918F917F916F9115
:103BB0005F914F913F912F910F900FBE0F901F90EB
:103BC00018951F920F920FB60F9211242F933F93C7
:103BD0004F935F936F937F938F939F93AF93BF9315
:103BE000CF93DF93EF93FF93C091E900CF70809163
:103BF000EC00D82FD17080FDD0E81092E9008091C0
:103C0000F000877F8093F00078940E94251E109228
:103C1000E9008091F00088608093F000CD2BCF7098
:103C2000C093E900FF91EF91DF91CF91BF91AF91E8
:103C30009F918F917F916F915F914F913F912F91C4
:103C40000F900FBE0F901F9018951F93CF93DF9387
:103C5000CDB7DEB7AA970FB6F894DEBF0FBECDBFC3
:103C6000E6E8F2E08091F100819322E0EE38F2077D
:103C7000C9F70E9490198091E80083FF2EC18091BE
:103C8000860290918702492F50E04A30510508F092
:103C900024C1FA01EE59FF4F0C94B51F803821F072
:103CA000823809F01AC108C0809182029091830283
:103CB000992389F082600FC080918A028F708730CB
:103CC00008F00BC18093E9008091EB0085FB882709
:103CD00080F91092E9009091E800977F9093E800B6
:103CE0008093F1001092F100D1C0282F2D7F09F0B0
:103CF000F4C0882319F0823061F0EFC0809188020F
:103D0000813009F0EAC0933009F080E080938302AB
:103D10002EC08091880281112AC080918A028F7002
:103D20002FEF280F263008F0D8C08093E9002091AB
:103D3000EB0020FF1CC0933021F48091EB008062E7
:103D400014C09091EB0090619093EB0021E030E083
:103D5000A90102C0440F551F8A95E2F74093EA007B
:103D60001092EA008091EB0088608093EB00109243
:103D7000E9008091E800877F8093E8000E94421C60
:103D8000ACC08111AAC0109188021F778091E30016
:103D90008078812B8093E3008091E800877F809377
:103DA000E8000E94421C8091E80080FFFCCF8091D7
:103DB000E30080688093E300111102C082E001C03B
:103DC00083E08093850289C08058823008F085C0E6
:103DD00080918802909189028C3D53E0950779F596
:103DE00083E08A838AE289834FB7F894DE011396D1
:103DF00020E03EE051E2E32FF0E050935700E491E1
:103E000020FF03C0E295EF703F5FEF708E2F90E0D0
:103E1000EA3010F0C79601C0C0968D939D932F5F36
:103E2000243149F74FBF8091E800877F8093E800F5
:103E30006AE270E0CE0101960E944E1B16C06091AE
:103E40008A0270918B02AE014F5F5F4F0E94921AFF
:103E5000BC01892B09F441C09091E800977F9093B1
:103E6000E80089819A810E94AC1B8091E8008B77E1
:103E70008093E80032C0803881F58091E800877F28
:103E80008093E800809181028093F1008091E800A6
:103E90008E7772CF811121C0809188029091890222
:103EA00099270297D4F48091E800877F8093E800F7
:103EB00080918802809381020E94421C809181023D
:103EC000811106C08091E30087FD02C081E001C03E
:103ED00084E0809385020E947C198091E80083FF32
:103EE0000AC08091E800877F8093E8008091EB0012
:103EF00080628093EB00AA960FB6F894DEBF0FBEE7
:103F0000CDBFDF91CF911F9108950895CF938091F8
:103F100085028823A1F0C091E900CF709091EC0058
:103F2000892F817090FD80E8C82B1092E900809164
:103F3000E80083FD0E94251ECF70C093E900CF9159
:103F4000089597FB072E16F4009407D077FD09D04B
:103F50000E94BB1F07FC05D03EF4909581959F4FB2
:103F60000895709561957F4F0895EE0FFF1F05909E
:103F7000F491E02D0994AA1BBB1B51E107C0AA1FB5
:103F8000BB1FA617B70710F0A61BB70B881F991FFA
:103F90005A95A9F780959095BC01CD010895FB0134
:103FA000DC0104C08D910190801921F441505040F2
:103FB000C8F7881B990B0895F999FECF92BD81BD72
:103FC000F89A992780B50895A8E1B0E042E050E062
:103FD0000C941020262FF999FECF92BD81BDF89A3E
:103FE000019700B4021639F01FBA20BD0FB6F8943D
:103FF000FA9AF99A0FBE08950396272F0E94EB1F95
:104000000E94EA1F252F0E94EB1F242F0C94EB1F08
:104010000196272F0E94EB1F0C94EA1FDC01CB01B5
:10402000FC01F999FECF06C0F2BDE1BDF89A3196C8
:1040300000B40D9241505040B8F70895F894FFCF66
:10404000C8000002280850011E0A1401C018E31815
:10405000C41853194F19C31801E200E900EA00B56A
:1040600000B600B700CD008301CC008A0192019414
:10407000012102230224022502260227022A02B37A
:1040800000B4006F007000818283E200E900EA0062
:10409000B500B600B700CD008301CC008A019201C3
:1040A00094012102230224022502260227022A0269
:1040B000B300B4006F007000818283919094F5F496
:0640C000F63534C6F700DE
:00000001FF
